BL51 BANKED LINKER/LOCATER V5.03                                                        04/25/2016  21:50:31  PAGE 1


BL51 BANKED LINKER/LOCATER V5.03, INVOKED BY:
C:\KEIL\C51\BIN\BL51.EXE led.obj TO led RAMSIZE (256)


MEMORY MODEL: SMALL


INPUT MODULES INCLUDED:
  led.obj (LED)
  C:\KEIL\C51\LIB\C51S.LIB (?C_STARTUP)
  C:\KEIL\C51\LIB\C51S.LIB (?C?SLCMP)


LINK MAP OF MODULE:  led (LED)


            TYPE    BASE      LENGTH    RELOCATION   SEGMENT NAME
            -----------------------------------------------------

            * * * * * * *   D A T A   M E M O R Y   * * * * * * *
            REG     0000H     0008H     ABSOLUTE     "REG BANK 0"
            DATA    0008H     0008H     UNIT         ?DT?LED
            IDATA   0010H     0001H     UNIT         ?STACK

            * * * * * * *   C O D E   M E M O R Y   * * * * * * *
            CODE    0000H     0003H     ABSOLUTE     
            CODE    0003H     00ECH     UNIT         ?PR?MAIN?LED
            CODE    00EFH     0016H     UNIT         ?C?LIB_CODE
            CODE    0105H     000CH     UNIT         ?C_C51STARTUP



OVERLAY MAP OF MODULE:   led (LED)


SEGMENT
  +--> CALLED SEGMENT
---------------------
?C_C51STARTUP
  +--> ?PR?MAIN?LED



SYMBOL TABLE OF MODULE:  led (LED)

  VALUE           TYPE          NAME
  ----------------------------------

  -------         MODULE        LED
  C:0000H         SYMBOL        _ICE_DUMMY_
  D:0090H         PUBLIC        P1
  D:00B0H         PUBLIC        P3
  D:00A8H         PUBLIC        IE
  D:00B8H         PUBLIC        IP
  C:0003H         PUBLIC        main
  D:0098H         PUBLIC        SCON
  D:0088H         PUBLIC        TCON
  D:00C8H         PUBLIC        T2CON
BL51 BANKED LINKER/LOCATER V5.03                                                      04/25/2016  21:50:31  PAGE 2


  D:0008H         PUBLIC        i
  D:000AH         PUBLIC        j
  D:000CH         PUBLIC        k
  D:000EH         PUBLIC        x
  D:00D0H         PUBLIC        PSW
  -------         PROC          MAIN
  C:0003H         LINE#         7
  C:0003H         LINE#         8
  C:0003H         LINE#         9
  C:0003H         LINE#         10
  C:0003H         LINE#         11
  C:0008H         LINE#         12
  C:0008H         LINE#         13
  C:0020H         LINE#         14
  C:0042H         LINE#         15
  C:0050H         LINE#         16
  C:0058H         LINE#         17
  C:0058H         LINE#         18
  C:005CH         LINE#         19
  C:0060H         LINE#         20
  C:0060H         LINE#         22
  C:0063H         LINE#         23
  C:0084H         LINE#         25
  C:0089H         LINE#         26
  C:0089H         LINE#         27
  C:0090H         LINE#         28
  C:00A9H         LINE#         29
  C:00CBH         LINE#         30
  C:00D9H         LINE#         31
  C:00E4H         LINE#         32
  C:00E4H         LINE#         33
  C:00E8H         LINE#         34
  C:00ECH         LINE#         35
  C:00ECH         LINE#         36
  -------         ENDPROC       MAIN
  -------         ENDMOD        LED

  -------         MODULE        ?C?SLCMP
  C:00EFH         PUBLIC        ?C?SLCMP
  -------         ENDMOD        ?C?SLCMP

Program Size: data=17.0 xdata=0 code=273
LINK/LOCATE RUN COMPLETE.  0 WARNING(S),  0 ERROR(S)
